:020000021000EC
:10F800000C9446FC0C9463FC0C9463FC0C9463FC19
:10F810000C9463FC0C9463FC0C9463FC0C9463FCEC
:10F820000C9463FC0C9463FC0C9463FC0C9463FCDC
:10F830000C9463FC0C9463FC0C9463FC0C9463FCCC
:10F840000C9463FC0C9463FC0C9463FC0C9463FCBC
:10F850000C9463FC0C9463FC0C9463FC0C9463FCAC
:10F860000C9463FC0C9463FC0C9463FC0C9463FC9C
:10F870000C9463FC0C9463FC0C9463FC0C9463FC8C
:10F880000C9463FC0C9463FC0C9463FC11241FBE69
:10F89000CFEFD0E1DEBFCDBF11E0A0E0B1E0E8E9FD
:10F8A000FFEF01E00BBF02C007900D92A430B1073B
:10F8B000D9F712E0A4E0B1E001C01D92A634B1076F
:10F8C000E1F70C948EFF0C9400FC0F92AF93BF9362
:10F8D000CF93DF93EF93FF93FC01EA01DB01D8950F
:10F8E000099231961197D9F7FF91EF91DF91CF915E
:10F8F000BF91AF910F9008950F921F920F931F9396
:10F90000AF93BF93CF93DF93EF93FF93FC01EA0193
:10F91000DB0110E00990199001E04CD0329612976B
:10F9200011F01250B9F7FC0103E044D005E042D0D9
:10F9300000E011E0800F911F109759F7FF91EF91B0
:10F94000DF91CF91BF91AF911F910F911F900F90B9
:10F9500008950F931F93EF93FF93FC0103E02AD0C8
:10F9600000E011E0E00FF11FE617F707B9F7FF918C
:10F97000EF911F910F9108950F930F9222D0082EAF
:10F9800009E018D00F900F9108950F930F92EF9305
:10F99000FF9317D0FC0160936800C895802DFF91FC
:10F9A000EF910F900F9108950F930BD001E102D0CA
:10F9B0000F910895E199FECF00936800E895FFFF4D
:10F9C00000000091680000FDFCCF089588E089B92F
:10F9D0008AB188618AB908958AB1877E8AB9089503
:10F9E0008CB95E9BFECF5E9A08958CB199270895DD
:10F9F0008BB19927807890700895EF92FF920F93C2
:10FA00001F93CF93DF937B01C0E0D0E0C617D707E9
:10FA100070F48C010E94F8FC8823E1F30E94F5FC4D
:10FA2000F80181938F012196CE15DF0598F381E0CF
:10FA300090E0DF91CF911F910F91FF90EF9008958B
:10FA4000EF92FF920F931F93CF93DF937C018B0173
:10FA5000C0E0D0E0C017D10738F4F70181917F01F1
:10FA60000E94F0FC2196F6CF81E090E0DF91CF91EB
:10FA70001F910F91FF90EF900895EF92FF920F93D7
:10FA80001F93CF93DF937C0100E010E00817190764
:10FA900088F4C0E0D0E000000E94F8FC882351F414
:10FAA000219687E0C03DD807B0F30F5F1F4F0E15BA
:10FAB0001F0578F3DF91CF911F910F91FF90EF9089
:10FAC00008950E94ECFC0E9400000895DF92EF92DE
:10FAD000FF920F931F93CF93DF93CDB7DEB721979C
:10FAE000DEBFCDBF8C017B011982D98061E070E05F
:10FAF000CE01860F971F0E94FDFC89818B31B1F7E3
:10FB000061E070E0C8010E94FDFC61E070E0CE01A0
:10FB1000860F971F0E94FDFC89819927182F0027C7
:10FB200061E070E0CE01860F971F0E94FDFC898185
:10FB3000080F111D61E070E0CE01860F971F0E9433
:10FB4000FDFC89818E30B9F4C8010196BC01C70162
:10FB50000E94FDFC98018FEF0F3F180779F0F70125
:10FB600081917F01D82621503040FFEF2F3F3F0782
:10FB7000B1F7DD2019F080E090E001C0C8012196C6
:10FB8000DEBFCDBFDF91CF911F910F91FF90EF901E
:10FB9000DF900895CF92DF92FF920F931F93CF9340
:10FBA000DF93182FEB016A018BE10E94F0FC4BE11F
:10FBB000F42E812F0E94F0FCF1260D2F1127802FAB
:10FBC0000E94F0FCF0268C2F0E94F0FCFC268EE0B8
:10FBD0000E94F0FC8EE0F82621978FEFCF3FD807E8
:10FBE00059F0F60181916F01F8260E94F0FC2197EF
:10FBF000FFEFCF3FDF07A9F78F2D0E94F0FCDF91C9
:10FC0000CF911F910F91FF90DF90CF90089599278A
:10FC10008139910559F08239910524F48039910593
:10FC200029F008C08239910519F004C082E003C0B0
:10FC300087E001C080EC99270895BF92CF92DF92B0
:10FC4000EF92FF920F931F93CF93DF93B82E8B0108
:10FC5000FB018081C82FDD27C231D10509F46DC0B9
:10FC6000C331D105DCF4C330D10509F44DC0C43033
:10FC7000D10544F4C130D10579F1C230D10509F480
:10FC80004AC018C1C630D10509F44AC0C630D105F2
:10FC90000CF410C160970CF40DC154C0C531D105EE
:10FCA00009F4DCC0C631D10544F4C331D10509F4EF
:10FCB0007CC0649709F449C0FDC0CA31D10509F47C
:10FCC000EBC0CB31D10524F4669709F4AEC0F2C085
:10FCD0006B9709F4D8C0EEC0FB01118288E08283E3
:10FCE00081E4838386E5848382E5858389E4868352
:10FCF00083E5878380E580878FE5818782E382873C
:10FD0000AB016BE070E0DCC0FB0181810E9407FE6B
:10FD1000F801828301C0FB011182A801BE01D0C09D
:10FD2000FB0183819927982F88272481820F911DB9
:10FD3000909345028093440206C060E070E0CB01DE
:10FD40000E94A9FCF8011182B8C0FB0181819927AA
:10FD5000D82FCC2782819927C82BD92B8091440298
:10FD60009091450297FF03C081E08BBF01C01BBE8D
:10FD7000F8011182C8010296209144023091450297
:10FD8000AC01BE01C901880F991F0E9465FCF801F2
:10FD9000EC0FFD1F12829E0136952795809144023B
:10FDA00090914502820F931F53C0FB0181819927D7
:10FDB000D82FCC2782819927C82BD92B8091440238
:10FDC0009091450297FF03C081E08BBF01C01BBE2D
:10FDD000CC24DD24CC16DD06D8F4FAE0EF2EF12C8D
:10FDE000E00EF11E8091440290914502880F991F08
:10FDF000A70160E071E08C0D9D1D0E947CFC80E0FD
:10FE000091E0C80ED91EE80EF91ECC16DD0650F39F
:10FE10000E94D4FCF8011182D695C79580914402C6
:10FE2000909145028C0F9D1F29C0FB01818199276C
:10FE3000D82FCC2782819927C82BD92B1182EC0F80
:10FE4000FD1F128280914402909145028C0F9D1FEC
:10FE5000909345028093440223965FCFFB018181FA
:10FE60009927382F222782819927282B392B118215
:10FE70008091440290914502820F931F9093450216
:10FE8000809344021AC0FB0111828481E82FFF276E
:10FE9000E050FF4F808107C0FB01118269E081E0E3
:10FEA00090E00E94C5FCF80182831382A80164E0FF
:10FEB00070E006C089ECF8018183A80162E070E07F
:10FEC0008B2D0E94CAFDDF91CF911F910F91FF9062
:10FED000EF90DF90CF90BF900895CF93DF93CDB791
:10FEE000DEB72197DEBFCDBF69E081E090E00E94E0
:10FEF000C5FC992784FF09C08F7E0E94BCFC05C009
:10FF000064E071E089810E941DFE64E071E0CE0131
:10FF100001960E9466FD892B99F3F7CFCFEFD0E1D0
:10FF2000DEBFCDBFCEE1F894AEEFBFE00E94C3FFCD
:10FF3000802D843B79F4AFEFBFE00E94C3FF802D9A
:10FF4000833C41F4ADEFBFE00E94C3FF802D9927B1
:10FF500080936F000E94E6FC0E94F5FC84E690E02E
:10FF60000E943DFD0E94F8FC882319F00E946DFF5D
:10FF700004C0C150C8BBCC2389F70E9461FD80E05A
:10FF800090E00C94CBFFE199FECFBFBBAEBBE09AF3
:08FF900011960DB20895FFCF98
:04FF98001E970200AE
:040000031000F800F1
:00000001FF
